S00F0000526563697665722E7372656345
S11300000C942A000C9447000C9447000C9447006D
S11300100C9447000C9447000C9447000C94470040
S11300200C9447000C9448010C9447000C9447002E
S11300300C9447000C9447000C9447000C94470020
S11300400C9447000C9447000C9447000C94470010
S11300500C94470011241FBECFE5D4E0DEBFCDBF12
S113006010E0A0E6B0E0ECE3F7E002C005900D92EA
S1130070A436B107D9F710E0A4E6B0E001C01D92A0
S1130080A636B107E1F70E9441030C949C030C943B
S1130090000080916200909163008630910509F41C
S11300A041C086E090E0909363008093620088E70B
S11300B090E090936100809360008FE39CE9019746
S11300C0F1F700C00000409162005091630081E0AC
S11300D06AE00E94E4028FEF96E1A1E18150904032
S11300E0A040E1F700C000008CE390E09093610031
S11300F0809360008FEF96E1A1E181509040A04091
S1130100E1F700C0000084EB90E0909361008093DD
S113011060008FEF96E1A1E181509040A040E1F7AB
S113012000C0000008958998809162009091630056
S11301308330910541F4819B06C00E946E020E94A7
S113014049000E94570280916200909163008230BE
S1130150910559F4819B09C00E946E0281E06AE016
S113016048E00E94E4020E945702B7992EC0809191
S11301706200909163008230910539F586E090E049
S113018090936300809362008FEF91E1AAE781501E
S11301909040A040E1F700C000008FEF91E1AAE792
S11301A081509040A040E1F700C000008FEF91E142
S11301B0AAE781509040A040E1F700C0000083E02E
S11301C090E090936300809362000895CF930E941F
S11301D0570202C00E9493000E9464028823D1F750
S11301E00E946902882341F08A3031F0803F09F08F
S11301F045C002C00E9493000E9464028823D1F784
S11302000E946902C82F02C00E9493000E946402E7
S11302108823D1F7C13091F50E946902843051F0EE
S1130220853018F48130B9F419C0853031F0873045
S113023091F40AC082E090E002C083E090E09093E1
S11302406300809362000AC00E946E020E9449000B
S11302500E94570213C00E946E0210C00E946E02D8
S11302608FE39CE90197F1F700C000004091620020
S11302705091630081E06AE00E94E402CF91089506
S113028085E083BF88E582BF1CBE81E089BF0895F5
S11302901F920F920FB60F9211242F933F938F93B7
S11302A09F9388E582BF80916200909163008230C1
S11302B0910541F480916400909165008333910528
S11302C034F11DC0809162009091630083309105E8
S11302D041F4809164009091650086309105BCF0F2
S11302E00EC080916200909163008630910579F48C
S11302F080916400909165008230910544F088B348
S113030091E0892788BB1092650010926400809167
S11303106400909165000196909365008093640059
S1130320B99AC19A8FEA94E00197F1F700C00000EE
S113033080E090E005C025E12A95F1F700000196E0
S1130340209160003091610082179307A4F3C19853
S11303509F918F913F912F910F900FBE0F901F90FF
S11303601895949840E120E030E097FF02C0969AF7
S113037001C09698220F331F83992160959A880FA4
S1130380991F00C000009598415079F7949AC901CB
S1130390089581B3806781BB949A8FEF90E7A2E0C0
S11303A081509040A040E1F700C0000080EE90EC46
S11303B00E94B10187ED90E80E94B1018BEA92ECB2
S11303C00E94B10181E89AEC0E94B10180E090EEB4
S11303D00E94B10180E098EC0E94B10187EF94EC97
S11303E00E94B1010895282F30E075E0220F331FD9
S11303F07A95E1F7307050E047705070242B352B1C
S11304003469862F90E083709070E3E0880F991F21
S1130410EA95E1F7822B932B0E94B101089580366F
S1130420910538F02FE08034920728F08FE39FE0A5
S113043002C080E690E0906A0E94B101089522E033
S113044087399207F8F09C0140E050E065E188317B
S1130450960768F460E678EA80E090E00E94810301
S1130460C90101978068966C0E94B10108956CEFF0
S113047072E485E090E00E945F03C9010197966CE5
S11304800E94B101089590E087709070986970E0BF
S1130490F4E0660F771FFA95E1F77070862B972BBF
S11304A00E94B10108959498839BFECF089588EC2F
S11304B092E80E94B10181E89AEC0E94B10183E8BC
S11304C09AEC0E94B1010895949881E0839980E0A8
S11304D0089580E090EB0E94B101089588E092E8CD
S11304E00E94B1010895FF920F931F93CF93DF935E
S11304F0182F092FF62E88E392E80E94B1010E947A
S113050053028AEA98EB0E94B1010E9453028AEADC
S113051098EB0E94B1010E9453028AEA98EB0E9470
S1130520B1010E9453028DE298EB0E94B1010E9436
S1130530530284ED98EB0E94B101C12FD02F08C063
S11305400E945302299130E0C901986B0E94B101C5
S11305508C2F811B8F15A0F30E94530288E092E830
S11305600E94B101DF91CF911F910F91FF900895E7
S1130570FF920F931F93CF93DF93182F092FF62E1B
S113058088EC92E80E94B10181E89AEC0E94B101E2
S113059083E89AEC0E94B101C12FD02F07C00E94BA
S11305A0530280E090EB0E94B10189938C2F811B50
S11305B08F15A8F388E092E80E94B101DF91CF91F2
S11305C01F910F91FF9008951F93CF93DF9300D055
S11305D0CDB7DEB7182F88E392E84A8369830E9477
S11305E0B1010E9453028AEA98EB0E94B1010E9471
S11305F053028AEA98EB0E94B1010E9453028AEAEC
S113060098EB0E94B1010E9453028DE298EB0E9484
S1130610B1010E94530284ED98EB0E94B1010E9443
S11306205302812F90E0986B0E94B1010E94530203
S11306306981862F90E0986B0E94B1010E94530259
S11306404A81842F90E0986B0E94B1010E9453026A
S113065080E098EB0E94B1010E94530288E092E886
S11306600E94B1018FEF90E7A2E081509040A0403A
S1130670E1F700C000000F900F90DF91CF911F9120
S113068008950E94C90180E296E00E940F0281E071
S113069060E047E00E94F30180E895E20E941F02B7
S11306A080E066E00E9443020E944001B89ABF982D
S11306B0C79ABD9AC59878940E94E600FDCFA1E23E
S11306C01A2EAA1BBB1BFD010DC0AA1FBB1FEE1FC8
S11306D0FF1FA217B307E407F50720F0A21BB30B13
S11306E0E40BF50B661F771F881F991F1A9469F78F
S11306F060957095809590959B01AC01BD01CF01EB
S1130700089597FB092E05260ED057FD04D0D7DF98
S11307100AD0001C38F450954095309521953F4FF0
S11307204F4F5F4F0895F6F79095809570956195BA
S10F07307F4F8F4F9F4F0895F894FFCF28
S107073CB4000200FF
S9030000FC
